:020000020000FC
:100000009AC461C01895189509945DC03AC01895B6
:1000100042C018951895E5C018951895189518952B
:10002000189572C01895697A40744042405B0290FE
:10003000FFFF7F0000B99FB68A9409F4E5E29FBEF6
:1000400018959FB68A949FBE189520FD939A21FD1E
:10005000949A22FD959AE1E3832C24BC1895A895E7
:1000600018958F12EECFA89511FDEFCFE0916500A6
:10007000852C20FD939821FD949822FD959844BCF1
:1000800018959FB640916300415008F40E7F40934D
:1000900063009FBE18959FB64091640043954093BE
:1000A00064004F7019F4BB2019F0BA949FBE1895E4
:1000B00040916600439540936600409167004395E8
:1000C00040936700F3CF46B557B59EB496FE0DC07A
:1000D0009FB65A5659BD48BD41E84EBD48E048BF9D
:1000E0009FBE18959FB6BB240BC098B693FCFACF61
:1000F0009FB63A0148B559B55659641A750A106148
:1001000041EC4EBD9FBE18959FB641B1403669F196
:100110004038B1F1403A69F1483A41F0483B79F052
:10012000483F11F04F1321C045ED20C067FC0DC0C2
:10013000F3B94AEF10FD4FEF40937D0016C067FC06
:1001400007C040917D0043B9F6CF4CE840937F0053
:100150005E2FE0917F004191E0937F0043B9E43945
:10016000E52F09F002C045E801C045EC46BF9FBE3F
:10017000189540917E004F131461F0937E00F5CFE7
:1001800040917E00439540937E00413019F473B056
:100190006F2EEBCF423011F463B0E7CF433021F440
:1001A00043B1423001F7E1CF4A3061F05E2FE9E818
:1001B000E40F43B14083E52F50919300540F5093C7
:1001C0009300D3CF43B150918D0056FD006157FD90
:1001D0000062451B50E9450F50938D0040939300FA
:1001E000C4CF9FB64CB1453F59F006FF0DC030F467
:1001F000509180005A9531F4742E18610F7B04C021
:10020000006451E0509380009FBE189590E578EC13
:10021000A39AC29A939A1ED0E1F7A398089594E600
:1002200074EBA29AC19A949A15D0E1F7A298089516
:1002300098E770EA929A959A0DD0E1F708959CE8B4
:100240007CE8A39AA29AC19A939A04D0E1F7A29863
:10025000A3980895F2BF82B78032E8F362B3677C57
:1002600062BB9298C298C19860E1F2BFA89582B72C
:100270008717E8F36A95C9F79A95089500D000D0DA
:1002800000D09FE060E1F2BF81E088BFA89588B709
:1002900080FFFDCF6A95B9F79A95A1F708958091EF
:1002A00084009091850089569A4739F0C4E8D0E0DF
:1002B000E6E285918993C439E1F70895F894EF93C4
:1002C000F5DFEF91789408958091600081BF0F7DF4
:1002D000C4E8D0E080E890E0A895E199FDCF67B749
:1002E00060FDFACFC43981F09FBB8EBB0196E09AC6
:1002F0006DB317F06993F0CF79917DBBF894E29AD2
:100300006713E19A7894E8CFBCDF8FEF81BF08953F
:10031000000C111CAA1C8A95D9F70895869FA12C60
:10032000969FA00CC11DDF1F879FA00CC11DDF1F62
:10033000979FC00DD11D089513FD4AC012FD3AC00C
:1003400013FD46C012FD36C01F76C30184369F07D9
:1003500008F40895C0917B00D0917C008C1B9D0B0C
:1003600060F41068909581959F4F6091790070912D
:100370007A0007C0CC27DD2710C06091770070910C
:10038000780080589140B2F3C8E3D0E0C7DFC735AA
:1003900083E0D80710F0C7E5D3E0C0937500D09391
:1003A000760001FF03C082E0B82EA7C080E1B81636
:1003B000BF1E0895E3011F7E8091920080FB17F914
:1003C000CC0FC295209649F3CE016DE373E0DCCFEC
:1003D000D72D1F76C0E0D03001F3CE0160E074E08D
:1003E000D3CF80918A0090918B0080937B00909373
:1003F0007C006091860070918700681B790B14D097
:10040000809377009093780060918A0070918B00C0
:100410008091880090918900681B790B05D08093AA
:10042000790090937A0008956058714085E595E0D1
:100430000196A8959F3F890721F0C0EEDCEF6EDFA3
:10044000B9F70895F8948CB59DB56091640078B7BC
:100450007894903872FD6F1FC0916800D091690048
:10046000A0906A00809368009093690060936A008E
:1004700000906B0010906C0070916D00C0936B0049
:10048000D0936C00A0926D0080199109670B973092
:100490006F0728F480E097E060E0D694C79461305D
:1004A000A7E5B3E058F06230ACEAB1E038F0643070
:1004B00018F080E090E064E0A6EDD0E07D0180934C
:1004C0006E0090936F006093700066959795879586
:1004D000C0916800D0916900A0906A0070E435D0A6
:1004E000C0937100D0937200A092730049D014FDA4
:1004F00027CFC0917500D0917600CE15DF0508F0AA
:10050000E701CC15DD0508F0E60187E593E08C1BDB
:100510009D0BB1F02096B1F01D7F116016FF04C055
:10052000880F991FCC0FDD1F75E29F137BE1C095EB
:1005300080951E01F8942C017093650078940895BD
:100540001360F2CF1C7F71E3F2CF879FC10DDF1FD5
:10055000AF1E979FC00DD11DAF1E679FD00DA11C70
:10056000089580916E0090916F0060917000C0912D
:100570007100D0917200A09073000895F2DFE5DF62
:1005800079B7072E7B7E79BF70E1F894DBBDCABDD9
:1005900078BF8CB59DB5789401606091640078B7A0
:1005A000903872FD6F1FC81BD90BA60AA09263007A
:1005B0000AF40E7F09BE0895279670E1F8948CB571
:1005C0009DB5C80FD91FDBBDCABD78BFA09263001F
:1005D00001607894089514FDB3DE00FDFCCF08950A
:1005E000F5BD80E488BFEFE29298C298C19882B3CB
:1005F000877C82BB0895B09BF09366008091660073
:1006000085FF0895E0E0F894FCE185919491F0E095
:10061000789401960297A8F3F894F7BBF4BBF1BB6A
:1006200088E181BDF1BD8091600081BFE9CA82E5AA
:1006300082B985EC86BF0895A298A398D2DE84E59E
:1006400088BF89BFF0BD89E189B9549A86E880BD29
:100650008CB15F9A579AEBDF81EC8EBD89B78062CF
:1006600089BFBB24137EF0936600F0936700A895C2
:1006700014FD0AC0C0DF809167008837C1F78CE3A2
:1006800080936700D5DDF3CF57DEC0917500D09120
:100690007600209631F78AE0B81648F312FFF6BFCD
:1006A00013FF5498812F8C7019F089B78F7D89BF03
:1006B000C6DDC5DDC4DD94DF0D7FA29AA398F0935B
:1006C0006600F0936700A89514FD0CC0BB20D9F715
:1006D00092DF809167008E31B1F782DFD2DDA8DD35
:1006E0009EDDAACF04FDEADD05FDEEDD29DE2096C4
:1006F00031F3BB2021F374DF80B7886080BFA398FB
:10070000A298CEE8D0E06E010260B1D0F093740000
:1007100082E0B82E86E0809362008CE080936100D6
:1007200081E085BD17FD39C0A6D081E087B9379833
:10073000C29810FD929A9DD0379AF894287F226033
:1007400082B3959892B38913949A789494D080E068
:1007500087B93798929810FDC19A8BD081E087B9FC
:100760003798F894287F216082B3949892B38913C4
:10077000939A789480D0379AC19810FDC29A79D014
:1007800080E087B93798F894287F246082B39398E3
:1007900092B38913959A789438C06BD0379AF894AD
:1007A000287F216082B3959892B38913939A7894A5
:1007B00062D081E087B93798C29810FDC19A59D0AC
:1007C00080E087B93798F894287F226082B39398A5
:1007D00092B38913949A78944ED0379AC19810FDA9
:1007E000929A47D081E087B93798F894287F24609F
:1007F00082B3949892B38913959A78943CD080E010
:1008000087B93798929810FDC29A80916100803024
:1008100010FFC1F0E6012096B1F08C3038F48395DA
:1008200080936100629686ED90E005C01F7BA398DF
:100830006B9687E593E0C817D90710F06C0172CF6B
:100840006E0170CF38CF57CFEFE282B3877C82BB87
:10085000A39A4EC016FD03C0BC30A8F5A39AF0932E
:10086000610070917400715F16FD709374001064E4
:100870003FC01F7D01C0106280916200815050F026
:100880008093620016FF0CC0C0E0DFEFAF2E94DE55
:10089000A4E020C0EF3211F4E1E3A39816FD34C0C8
:1008A0007BE16CDE98DE73E369DE00FFCDCF14FDE3
:1008B00047DD68B1612765FDF8CF53DEA92F6F13BF
:1008C000AFEFAC3038F44DDEC80FD91FA61E58DE8E
:1008D000BBE001C0BA2F00FFBDCF14FD31DD68B110
:1008E000612765FD03C0AB17AF1FF5CFAA9599F738
:1008F000A9DD16FF70DE809162008F131E7FBF128C
:1009000008958F918F91D7CEC0E0D0E070E0A72EF0
:1009100080916100823030F47091740080E090E842
:1009200060E013DE49DE57DEC0E0D8EB7BE0A72EA7
:1009300043DEAFEFCFCF00240FBEEFE5F4E0FEBF04
:10094000EDBF0292E036F00509F4EEE1E015F005A6
:10095000C1F781B780936000A4B6F4BFF8BB86E00E
:1009600087BB80E385BBF4BB82E082BB8EE381BBA7
:1009700082E083BF81EC8EBDF5BD88E181BD88E05A
:1009800081BD7FDCA1DC8BDC52DE7894A0FAAF1253
:1009900026F43CDC44DC4CDC4FCEA2FE04C048DC38
:1009A00035DC006849CEA1FE02C049DC45CEF89492
:1009B000A3FE05C02BDC2ADC3BDC3ADCFBCF5EDC93
:1009C0004A2D58E040FF2BDC40FD39DC58DC4695D1
:0609D0005A95C1F7F4CFB7
:101C0000E4E0FFE5FEBFEDBF00E0ECEBFEE0C0E886
:101C1000D0E0A0E6B0E042E045BD5CEE539571F047
:101C200040EC04BD48BFA03619F0E8B6E6FC46C05B
:101C3000B099F9CF04BD48BFE8B6E6FCE1C1B09B5E
:101C4000FBCF04BD48BFE8B6E6FCE8CFB099FBCFB8
:101C500034B404BD48BFE8B6E6FCD2C1B09BFBCFAC
:101C600024B4022C030C802C07940694402C069478
:101C70008008809420943094409460EE83E084BC8B
:101C800048BFE8B6E6FCBCC1B09BFBCF84BC48BFF4
:101C9000E8B6E6FCC3CFB099FBCF0894E8B6E6FC03
:101CA00023C0B09BFBCFE8B6E6FCB8CFB099FBCF22
:101CB0008894E8B6E6FC18C0B09BFBCF43BC87E134
:101CC000C09AB89A34BC48BFE8B6E6FEFDCFC098CB
:101CD00024BC48BFE8B6E6FEFDCF8A9589F7C0E68A
:101CE000D0E060E081E00BC0679548F6815068F570
:101CF0005CEE0994CA17DB07D1F0699188E066951C
:101D0000C09A34BC48BFE8B610F0E7FC08BBE6FE5A
:101D1000FACFC09808F0C09A24BC48BFE8B610F0CB
:101D2000E7FC08BBE6FEFACF8A9549F7E3CFC09AF5
:101D300034BC48BFC0E8D0E0A0E6B0E0E8B6E7FEBB
:101D4000FDCFB89808BB6ACF80E060E898CFECEB95
:101D5000FEE0C0E8D0E0F8CF009000000090000066
:101D60000090000000900000009000000090000033
:101D70000090000000900000000000006B3121F78F
:101D8000562E3796E1CF962E56263496DDCF762EF8
:101D900056263496D9CF662E56263496D5CF6E3039
:101DA000B1F656263596D0CF69935626CF3584E0C6
:101DB000D80768F681E0681A700A09F43C96C4CF27
:101DC0006511C5CFC0E8D0E0699199918991FD0175
:101DD0007BE170839182028372E073837EE074837F
:101DE0006583068317966130A1F48BE0838388E0D6
:101DF0008D93EF01ECEDFFE185918D93E43EE1F7EA
:101E0000FE01819161918627EA17FB07D9F78D932F
:101E10009ECF6D3151F5792F90E0039683839283A5
:101E200003970D938A95E9F789916991603380074B
:101E300094E0790779F460878991803059F4699149
:101E400060308EE131F0613083E919F0623087E073
:101E500009F482870D93D5CF8017900709F5D990A3
:101E6000C9905601AA0CBB1CCCCF6330E1F06230A4
:101E700041F2603131F2613121F2663069F3623151
:101E8000F1F1833F73E0970758F4643109F166314B
:101E900069F127966531C1F16331F9F10000000065
:101EA00080EC8683AECF90398FE071F0913982E07B
:101EB00059F092398AE041F0943982E329F0903860
:101EC00080E011F0913861F78D9383E0838399CF9F
:101ED00049D0EF01F5018FD076FDFDCF65916D936F
:101EE0000197E1F75F01FE010D938BCF3BD011E02D
:101EF0003ED06DB36D930197D9F70D9382CF47D044
:101F0000000080E092E0689416E06FEF0EF06991B7
:101F10002ED00197D1F7E89474CF8F7F61E07F01D5
:101F2000F5010990199068D032960297D1F70F0108
:101F3000F501500163E0E03C7FE1F70719F058D06C
:101F4000F7015FCF0BD065E009D061E107D0F8CF92
:101F500077B770FDFDCFE199FECF0895F9DF67BF38
:101F6000E8950895039692838383039708953AD062
:101F7000DFBACEBA0894C01ED01E762FE09A6DB399
:101F8000671312FF08957DBBE29A1CBB08957F0181
:101F9000E0E0FEE063E0B0972FD0E9F76F01F701D2
:101FA0000895000000000000000000000000000094
:101FB0000000000000000000000000000000000021
:101FC000687474703A2F2F6769746875622E636F36
:101FD0006D2F73696D2D2F7467792F00415652490B
:101FE00053505F3277B770FDFDCFE199FECF089572
:101FF00003D065E001D061E1F5DF67BFE8950895A2
:00000001FF
